:020000040000FA
:1000000001288316003085000030860083128501A8
:1000100086019B019C019D010616061386120A1497
:100020008A1411230A108A100A148A141F230A1032
:100030008A1000309100053092000A148A140023BF
:100040000A108A10083085060A148A1411230A102F
:100050008A100A148A141C230A108A102C308C006F
:1000600037200A148A1419230A108A101928FF301D
:100070008D0002309300643094001B3095003330C3
:1000800096000A148A144A230A108A101D1C392863
:1000900000309100963092000A148A1400230A104E
:0C00A0008A108E0B39288D0B39280800BF
:1006000091099209920A0319910AF83090000000AA
:10061000900B072B00000000920A0319910F052B85
:1006200008001923222336239801990100303E2324
:1006300008001D11F8306B2B1D15C0306B2BA0303E
:100640009D106B2BB0309D146B2B1D1C2F2B0000AD
:100650001D109D1C2D2B50306B2B861308001D1474
:100660009D1C342B58306B2B8617080040306B2BA9
:1006700042306B2B44306B2B46306B2B9A00183872
:100680009B0019089C006D231A0809389B00180864
:100690009C006D2B1D1C502B000000305323282B79
:1006A000043053232F2B970030389B0016089C00F2
:1006B0006D23170821389B0015089C006D2317082F
:1006C00032389B0014089C006D23170823389B00C8
:1006D00013089C006D2B9B009C01061210309E009D
:1006E0009B1F86129B1B8616061706139C0D9B0DDF
:0806F0009E0B702B061608009A
:02400E00F13F80
:00000001FF
